:020000040000FA
:100000009E01BF28930005108510851083160510EA
:10001000851085100F308605831213089E182E2830
:100020003A308D009830A7203330920042201330B0
:100030008D008830A72042206430A6204220643002
:10004000A62022309200422028302D200C302D2076
:1000500006302D209E1413082E281E1492001E1CFC
:100060003C288510033C031C4128412015308D009D
:100070007C30A720031408001E14FE3C0319BA2884
:1000800085141E1C1E1005140F3086051208F03949
:1000900086040510920E1E1842283230A620031442
:1000A00008008F00220884002009812084138F0813
:1000B0000319BA28F03091000E0880389000F03013
:1000C00091030319910003198F030319BA280C082F
:1000D00092000D0893001630A62012088C00130819
:1000E0008D008A2003010C1820088E1F20088E081E
:1000F00003190301900F7E2880065C287F280000EA
:100100005F2884178005BA288001840AFF3E031DFA
:100110008428BA280D080C0403198C0A80300C1AA4
:100120008D060C198D068C188D060D0D8C0D8D0D00
:10013000BA288F018E00FF308E07031C8F07031C27
:10014000BA2803308D00E330A7209B288D01F43EB0
:100150008C008D09FE30031CB0288C070318AD28D5
:100160008C0764008D0FAD2800000C18B7280C1800
:10017000B9280800831303138312640008008B015D
:1001800083168501083086000C30840044308312C9
:100190008420051183160511323083129920FE3018
:1001A000022001300220FE30022080300220473041
:1001B00002206130022073300220FE300220C03065
:1001C0000220443002206530022074300220653065
:1001D000022063300220743002206F30022072301F
:1001E00002200B308F00B8309A20FE300220013000
:1001F0000220FE300220803002205630022065307E
:1002000002207230022073300220693002206F30E9
:1002100002206E30022020300220FE300220C0304A
:100220000220203002202030022020300220203006
:10023000022020300220313002202E3002203030C7
:10024000022003308F00E8309A20FE300220013077
:100250000220FE300220803002204230022079301D
:1002600002202030022052300220753002206930F6
:100270000220FE300220C0300220433002206130D4
:1002800002206230022072300220613002206C3085
:10029000022006308F000E309A206400861D9329BC
:1002A000FE30022001300220FE3002208030022089
:1002B0002A300220463002206F30022075300220A2
:1002C0006E300220643002202A300220FE300220EC
:1002D000C0300220213002202130022020300220B4
:1002E000473002206130022073300220203002208B
:1002F000213002206400861D932901308F002C30AC
:100300009A200430850683160511831201308F0070
:100310002C309A200630A2000130A00078308E00E8
:10032000643051207A2996309920FE300220013025
:100330000220051183160511FE3083120220803041
:10034000022053300220653002206E3002207330CC
:100350000220693002206E30022067300220FE3019
:100360000220C03002204E3002206F3002202030A8
:1003700002204730022061300220733002202030FA
:100380000220213002204D29FE30022001300220BF
:10039000FE300220803002202A3002204630022027
:1003A0006F300220753002206E300220643002204F
:1003B0002A300220FE300220C030022021300220EC
:1003C00021300220203002204730022061300220FC
:1003D00073300220203002202130022096309920F4
:1003E000043085068316051183124D296300F62912
:02400E00FD3F74
:00000001FF
